:100000000C946D000C94F0000C94F0000C94F00033
:100010000C94F0000C9447100C94F0000C94F00039
:100020000C94F0000C94F0000C94F0000C94F00090
:100030000C94F0000C94F0000C94F0000C94550A11
:100040000C94F0000C94F0000C942F0F0C948F0F74
:100050000C94F0000C94F0000C94F0000C94F00060
:100060000C94F0000C94F0000C94F0000C94F00050
:100070000C94F0000C94F0000C94F0000C94F00040
:100080000C94F0000C94F0000C94F000A218A51849
:10009000A818AB18AE18B518B818BB18BE18F618C3
:1000A0001B19201925192A192F1939194C194F19FB
:1000B00056196419D319D319D319D3197319791986
:1000C000821994199719A319D319A619AC19AF1944
:1000D000B519B819BE19C119C91985B7806885BF86
:1000E00080916C00806880936C00BF9ABE9AC7981C
:1000F000C69880EC85BFAF9AA79AAE9AA69A81EE71
:100100008093008380E4809301832FE785B7822367
:1001100085BF80E090E09D9B05C0019641F09D9BCE
:10012000F8CFFBCF019619F09D99F3CFFBCF85B7A0
:10013000806885BF85B3822385BB84B3822384BB5B
:10014000AE98A69887E089B98093990011241FBEC4
:10015000CFEFD0E1DEBFCDBF11E0A0E0B1E0E6EE31
:10016000F6E300E00BBF02C007900D92AA3DB10775
:10017000D9F712E0AAEDB1E001C01D92A333B10797
:10018000E1F78FEF9FEF9EBF8DBF8FEF9FEF835300
:1001900092408158914048F08FEF9EEF83539240F8
:1001A000BC0183E392E00E94EE060E94FA06892BCE
:1001B00059F0A7E0B2E0E1E2F1E089E001900D92B0
:1001C0008150E1F70E94160720E831E040E050E05E
:1001D00066E771E08AE291E00E94D4080C94000086
:1001E0000C9400000F931F93CF93DF93CDB7DEB72E
:1001F00064970FB6F894DEBF0FBECDBF8091F201B9
:100200009091F3010E946D1044E150E0BE016F5FD8
:100210007F4F0E944E118C010E94081521E0422F51
:1002200060E085E00E94ED122FEF44E060E087E09F
:100230000E94ED128091F2019091F3010E946D10E5
:10024000A801BE016F5F7F4F0E946111D7CFCF938E
:10025000DF93CDB7DEB724970FB6F894DEBF0FBE9D
:10026000CDBF80E091EEA0E0B0E089839A83AB83BC
:10027000BC830E94C01140E060E070E085E391E043
:100280000E94BB0160E071E087E391E00E94711081
:100290009093F3018093F2010E946D10AE014F5FC5
:1002A0005F4F61E071E00E94E1106091F201709196
:1002B000F30183E091E00E94D01081E00E941815C4
:1002C0002FEF44E060E087E00E94ED120E94F20010
:1002D00081E090E024960FB6F894DEBF0FBECDBF4C
:1002E000DF91CF91089580931B0108950E9404022D
:1002F00020E033E040E050E067E271E08CE191E023
:100300000E94D4088EEF0E948C050E943A050E943C
:10031000520520911B012F3FC1F395B79C7185B702
:10032000837E822B85BF85B7806285BF889585B720
:100330008F7D85BF85B7837E892B85BFE6CF0F93E1
:100340001F93CF93DF938C01C091DB01D091DC012F
:10035000209759F0B801CE0102960E94ED1A892B20
:1003600021F00990D881C02DF3CFCE01DF91CF913C
:100370001F910F910895EF92FF920F931F93CF93C8
:10038000DF93EC018FEFE82EF82E209709F161152D
:10039000710511F07D876C8741114E87CE01029661
:1003A0000E949F018C01892B99F4EB89FC8930977D
:1003B00021F0CE010995892B59F48091DB019091B0
:1003C000DC0199838883D093DC01C093DB01780141
:1003D000C701DF91CF911F910F91FF90EF9008958A
:1003E0008091F6019091F701A091F801B091F90187
:1003F0000196A11DB11D8093F6019093F701A09382
:10040000F801B093F901089580EF91E00E94870907
:1004100087B7826087BF0895CF93DF93EC011B827B
:100420001A82E091F401F091F5013097D9F0288516
:1004300039854A855B8580859185A285B385281796
:1004400039074A075B07D8F0281B390B4A0B5B0BAF
:10045000288739874A875B87FB83EA830190F0818D
:10046000E02DE3CFF983E883309711F0D383C28383
:10047000EA81FB81309761F0D183C0830DC0821B7C
:10048000930BA40BB50B80879187A287B387EACF24
:10049000D093F501C093F401DF91CF9108950FB689
:1004A000F8940F928091F6019091F701A091F801D4
:1004B000B091F9010F900FBEBC01CD0108958F924C
:1004C0009F92AF92BF92CF92DF92EF92FF920F93E3
:1004D000CF93DF936B017C015A01490180E190E0E9
:1004E0000E94EA05EC01892B39F10E944F02DC01E0
:1004F000CB018C0D9D1DAE1DBF1D2091DD013091E6
:10050000DE014091DF015091E001821B930BA40BAF
:10051000B50B88879987AA87BB8700FF05C01C8217
:100520001D821E821F8204C0CC82DD82EE82FF8289
:10053000BD86AC869F868E86CE01DF91CF910F91CE
:10054000FF90EF90DF90CF90BF90AF909F908F90F3
:100550000895CF92DF92EF92FF920F93CF93DF93A4
:100560006B017C01C701B6010E945F02EC0100979C
:1005700011F00E940C02CE01DF91CF910F91FF90FC
:10058000EF90DF90CF900895CF92DF92EF92FF929D
:100590000F931F93DC01CB016A017901BC01CD01EE
:1005A0000E94E709DC01CB019701A601BC01CD0146
:1005B0000E94A9021F910F91FF90EF90DF90CF90C2
:1005C0000895AF92BF92CF92DF92EF92FF920F9376
:1005D0005B016C016115710581059105D9F16CEF25
:1005E00071E08091FE019091FF010E94AE04E091C4
:1005F000FE01F091FF0183E08787E090FE01F0901B
:10060000FF0101E097014FE255E0C601B5010E94EC
:10061000C402F701968B858B892B19F00E94EA049E
:100620001BC0E091FE01F091FF018CEF91E0908FF3
:10063000878B8091FC019091FD019383828381E0FF
:1006400087878091FE019091FF019093FD01809337
:10065000FC0102C00E943A050F91FF90EF90DF90DD
:10066000CF90BF90AF900895CF93DF93EC01EA81D4
:10067000FB8188819981309719F09183808304C030
:100680009093F5018093F401E881F9813097A1F00E
:100690008A819B819383828380859185A285B3859E
:1006A000288539854A855B85820F931FA41FB51F56
:1006B00080879187A287B387CE010E947006DF9161
:1006C000CF910895EF92FF920F931F93CF93DF93F3
:1006D0000E944F029B01AC018091DD019091DE01EF
:1006E000A091DF01B091E00179018A01E81AF90ACD
:1006F0000A0B1B0B2093DD013093DE014093DF01D9
:100700005093E001C091F401D091F501209709F4D4
:1007100061C0E114F1040105110509F45BC088858D
:100720009985AA85BB85E816F9060A071B0760F4B8
:100730008E199F09A00BB10B88879987AA87BB8761
:10074000EE24FF24870108C0E81AF90A0A0B1B0BE4
:10075000188619861A861B8688859985AA85BB8581
:100760000097A105B10551F5EC85FD85309721F085
:100770006E857F85CE0109958C819D81AE81BF817B
:1007800088879987AA87BB870097A105B10521F4BF
:10079000CE010E94340312C0E091F401F091F50102
:1007A0000190F081E02DF093F501E093F401309792
:1007B00011F013821282CE010E940C02C091F4014A
:1007C000D091F501209731F0E114F10401051105F4
:1007D00009F0A5CFDF91CF911F910F91FF90EF907E
:1007E0000895EF92FF920F931F930E944F027B0197
:1007F0008C010E94E2099B01AC01C801B7010E9473
:10080000291BCA01B9011F910F91FF90EF90089524
:100810006F927F928F929F92AF92BF92CF92DF9210
:10082000EF92FF920F931F930E944F025B016C01A6
:100830000E94E2099B01AC01C601B5010E94291B7F
:1008400079018A010E94E2099B01AC01C801B7014C
:100850000E94F71ADC01CB01A81AB90ACA0ADB0AFE
:1008600088EE682E83E0782E812C912CC801B70188
:10087000A40193010E94F71A7B018C01C601B50106
:100880000E94F71A5B016C010E94E2099B01AC0116
:10089000C601B5010E94291BE20EF31E041F151F9D
:1008A000C801B7011F910F91FF90EF90DF90CF909B
:1008B000BF90AF909F908F907F906F900895CF934F
:1008C000DF93DC019B01EC01788F6F8B1D821C8212
:1008D0000FB6F8940F92EB01E881F9818FEFEF3FAB
:1008E000F80749F4E0E0F0E0ED018C819D8101968C
:1008F0009D838C8316C03097A1F00F900FBE828924
:10090000ED019A89981750F09F012E5F3F4F0280AA
:10091000F381E02D309711F08289F4CF0FB6F8946F
:100920000F92ED01FB83EA83F901B183A083EA8191
:10093000FB81309771F084819581892B51F08C81F6
:100940009D8124813581820F931F9D838C83158225
:1009500014820F900FBEDF91CF910895CF93DF9354
:100960009C01DB010FB6F8940F92ED91FC91119769
:100970000F900FBE8FEFEF3FF80749F1309739F135
:1009800082819381E217F307E9F40FB6F8940F928E
:1009900011969C938E9384819581892B59F0A28125
:1009A000B381109729F084819581ED019D838C831B
:1009B000158214820F900FBEF90113821282108EDD
:1009C000178A05C0DF011296FC01892BC9F6DF9159
:1009D000CF910895CF93DF93C091FA01D091FB019D
:1009E000209709F10FB6F8940F928C819D810F909A
:1009F0000FBE892BA1F0EF89F88D0FB6F8940F92F6
:100A00008C819D8101979D838C83808191810F9042
:100A10000FBE8F5F9F4F19F0CF010E94EF07099023
:100A2000D881C02DDDCF0E946203E091FE01F091DC
:100A3000FF018091FC019091FD01E817F90761F039
:100A40008785813011F482E087870FB6F8940F9282
:100A50000E9495080F900FBEDF91CF910895FB0182
:100A6000168A158A82E087876CEF71E0CF010E94B9
:100A70005F040895E091FE01F091FF01828193816E
:100A8000892B69F06CEF71E0CF010E94AE046CEF2E
:100A900071E08091FE019091FF010E945F040E942D
:100AA000EA040895E0910002F0910102309741F0CC
:100AB000838994890E9470061092010210920002AC
:100AC00008950F931F93CF93DF93C091FA01D091B4
:100AD000FB010AEF11E00E945205209781F08091FE
:100AE000FE019091FF0128813981C817D90721F4AF
:100AF000F8013183208303C08E01E901EECF80919C
:100B0000FE019091FF019093010280930002DF911A
:100B1000CF911F910F9108951F93CF93182FE091BC
:100B2000FE01F091FF01C2896CEF71E0CF010E94DC
:100B3000AE04E091FE01F091FF01128B1F3F49F0DE
:100B40006CEF71E08091FE019091FF010E945F04C3
:100B500002C00E946105E091FE01F091FF018091C9
:100B6000FC019091FD01E817F90719F481E08787EE
:100B700009C082E087870FB6F8940F920E9495080B
:100B80000F900FBE8C2F9927CF911F9108958FEF53
:100B90000E948C0508950F931F93CF93DF938C01D0
:100BA000C091FA01D091FB01209769F0B801CE0104
:100BB00006960E94ED1A892B11F4CE0106C0099009
:100BC000D881C02DF1CF80E090E0DF91CF911F91CF
:100BD0000F910895CF93DF93AC01C0E0D0E0DE0128
:100BE0008091E1019091E2014817590720F05FC020
:100BF000EF01DB0129C04A5F5F4F4430510510F41B
:100C000044E050E0E0910202F091030262E072E001
:100C1000309709F44CC0208131812417350760F0EA
:100C20002417350729F3209729F0888199812817FF
:100C3000390710F4EF01DB01BF016E5F7F4F0280C7
:100C4000F381E02D309739F7209789F1CA010A9690
:100C5000288139816A817B818217930770F4FE01B4
:100C6000E40FF51F241B350B3183208373836283CC
:100C700059834883ED93FC9302C06D937C938091DC
:100C8000E1019091E201E881F9818E1B9F0B909325
:100C9000E2018093E101EC0FFD1F34978FEE9EEB94
:100CA000ADEABEED80839183A283B3832296CE0109
:100CB000DF91CF9108950F931F93CF93DF938C0112
:100CC0000E94EA05EC01009729F0A80160E070E0BD
:100CD0000E94E31ACE01DF91CF911F910F910895E9
:100CE000EF92FF920F931F93CF93DF932EEFE22E9D
:100CF0002FEFF22EE80EF91ED7014D915C91E09195
:100D00000202F091030202E012E0309709F44BC0B6
:100D1000B701640F751F808191819F01280F391FD2
:100D20002E153F05D1F49C01240F351F31832083FC
:100D3000DF01A20FB31F82819381A817B90799F52C
:100D40008D919C911197280F391F31832083ED01DC
:100D50008A819B819383828326C0EE16FF06A0F4CE
:100D6000D801ED92FC926E177F0751F4840F951F06
:100D7000E70199838883828193819B838A8313C04F
:100D8000E701FB83EA830FC0E216F30618F48FEF46
:100D90009FEF1DC08F010E5F1F4F0280F381E02D7A
:100DA000309709F0B8CF309731F4E701FB83EA833D
:100DB000F801F182E0828091E1019091E201840FDB
:100DC000951F9093E2018093E10180E090E0DF9134
:100DD000CF911F910F91FF90EF900895FC016193C7
:100DE0007193CF010E94700608958091E101909166
:100DF000E201089543E150E064E072E080E090E0B9
:100E00000E9487089C01892B61F480910402833140
:100E100041F4809105028F3421F4809106028335DC
:100E200019F08FEF9FEF0895C901089583E1809332
:100E300004028FE48093050283E58093060243E178
:100E400050E064E072E080E090E00E948A08009741
:100E500011F08FEF9FEF0895CF93DF93AC01DB018B
:100E60000FB6F8940F92CD91DC9111970F900FBEB1
:100E70008FEFCF3FD80709F436C02097A1F18D89B5
:100E80009E892A813B818417950741F50FB6F89416
:100E90000F9211963C932E938C819D81892B81F02A
:100EA000EA81FB81309729F08C819D819583848331
:100EB00005C08FEF9FEF11969C938E931D821C822D
:100EC0000F900FBE82E08F876CEF71E0CE010E9421
:100ED0005F048FEF9FEF9E8B8D8B05C0DE01129616
:100EE000E901232B61F6DF91CF910895AF92BF9274
:100EF000CF92DF92EF92FF920F93CF93DF93EC01AB
:100F00005A016B010FB6F8940F92888199810F9066
:100F10000FBE8F5F9F4F51F40FB6F8940F92198256
:100F200018820F900FBE0E943A053CC06CEF71E032
:100F30008091FE019091FF010E94AE04BE0180915C
:100F4000FE019091FF010E945F04E091FE01F0918B
:100F5000FF0183E08787E090FE01F090FF01A1147C
:100F6000B104C104D10461F001E09E014CE257E0FC
:100F7000C601B5010E94C402F701968B858B03C0A0
:100F8000F701168A158A0E94EA04E091FE01F091A9
:100F9000FF01858996892FEF8F3F920719F4168AF2
:100FA000158A02C080E090E0DF91CF910F91FF9011
:100FB000EF90DF90CF90BF90AF900895FC010FB6F7
:100FC000F8940F92808191818F5F9F4F11F411826D
:100FD00010820F900FBECF010E9476070895CF9325
:100FE000DF93DC010FB6F8940F92CD91DC9111974D
:100FF0000F900FBE8FEFCF3FD80709F43AC020976C
:1010000071F10FB6F8940F92EA81FB811196FC936F
:10101000EE938C819D81892B71F0309729F08C8122
:101020009D819583848305C08FEF9FEF11969C93DC
:101030008E931D821C820F900FBE8D899E89009712
:1010400021F00E9434031E8A1D8A82E08F876CEF94
:1010500071E0CE010E945F0481E090E00CC00FB609
:10106000F8940F928FEF9FEF11969C938E930F90B1
:101070000FBE80E090E0DF91CF9108950F931F9312
:101080000E94EF078C010E943A05C8011F910F9141
:1010900008950F931F93CF93DF93EC0100E010E0CE
:1010A0000FB6F8940F92888199810F900FBE2FEFA1
:1010B0008F3F920741F40FB6F8940F92198308837B
:1010C0000F900FBE13C0892B89F0CE010E94EF074D
:1010D000080F191F0FB6F8940F92888199810F900D
:1010E0000FBE009719F08F5F9F4F79F7C801DF910E
:1010F000CF911F910F9108950F931F930E9449085C
:101100008C010E943A05C8011F910F9108950E9419
:10111000BE0E08950E94CE0E08959F918F910F905C
:101120000BBE0F900FBE1F9018952F923F924F92BB
:101130005F926F927F928F929F92AF92BF92CF9267
:10114000DF92EF92FF920F931F93CF93DF938DB7B0
:101150009EB7E091FE01F091FF01918B808BE091B1
:10116000FC01F091FD01F093FF01E093FE0181E0AD
:101170008787E091FE01F091FF01808991898DBF01
:101180009EBFDF91CF911F910F91FF90EF90DF9065
:10119000CF90BF90AF909F908F907F906F905F9017
:1011A0004F903F902F900895AF92BF92CF92DF92D1
:1011B000EF92FF920F931F93CF93DF937C016B010C
:1011C0005A01E901C90149960E94EA05FC0100970C
:1011D00009F478C08C010C0F1D1FB80167507040D6
:1011E000A8014B515040C801069628E0D7010D9048
:1011F0007D01EC010992CE012150C1F7E8012E8753
:1012000041505040598B488B4F5F5F4FFC8BEB8BAD
:101210008FEE9EEBADEABEED80839183A283B38314
:1012200084839583A683B78380879187A287B387BA
:1012300084879587A687B78780E48A8B8D2D992729
:10124000FB018583C68280E8838322832483A18275
:101250008B2D992780832DE838E0832F9927EA0189
:101260008A8B2B8B8091FA019091FB01F80191837D
:1012700080831093FB010093FA01C2E0C787168AAE
:10128000158A108E178A6CEF71E0C8010E945F0406
:10129000E091FE01F091FF01309721F40FB6F89430
:1012A0000F925DCF8091FC019091FD01E817F90745
:1012B00041F0C7870FB6F8940F920E9495080F90DF
:1012C0000FBEC801DF91CF911F910F91FF90EF905A
:1012D000DF90CF90BF90AF9008951F93182F80910B
:1012E000E3019091E401A091E501B091E601BC0118
:1012F000CD0120EA3FE040E050E00E94291BE22FB0
:10130000F32F3197F1F71A95D1F71F910895BC018A
:1013100087B78D7F87BF80B7886080BF12BE82E0AD
:1013200083BF80B7992787709070892BD1F781E0B0
:1013300086BF0FB6F8940F9281E090E0A0E0B0E095
:10134000B6B7B170E9F3B6BF0894811D911DA11D18
:10135000B6B7B170C9F3BB270F900FBE27E0880F57
:10136000991FAA1FBB1F2A95D1F78093E301909381
:10137000E401A093E501B093E60187B78D7F87BFB5
:1013800080B7886080BF12BE89E083BF8FE181BFD4
:1013900080B7482F55274770507041155105C1F748
:1013A00082E086BF8FE291E00E94041A0895809146
:1013B000E3019091E401A091E501B091E601BC0147
:1013C000CD01089560E074E080E090E00895EF9230
:1013D000FF920F931F937B018C010E94E2099B01F6
:1013E000AC01C801B7010E94F71ADC01CB01BC01B6
:1013F000CD0128EE33E040E050E00E94291B21158A
:1014000031054105510521F421E030E040E050E094
:10141000CA01B9011F910F91FF90EF9008959C01AF
:10142000FB0160E070E087B7482F5527427050708D
:1014300087B78D7F87BF20313105C1F0213131055C
:101440003CF42115310571F02130310561F024C0E3
:101450002231310541F12231310514F120323105BB
:10146000B1F01AC0AB0182E086BF18C006B601FE1B
:1014700005C081E090E09183808302C07183608326
:101480004115510559F080819181806802C08EE03C
:1014900090E09183808302C06FEF7FEF452B19F0BE
:1014A00087B7826087BFCB0108951F920F920FB656
:1014B0000F9211242F933F934F935F936F937F93DA
:1014C0008F939F93AF93BF93EF93FF938FE291E03E
:1014D0000E94F919FF91EF91BF91AF919F918F9168
:1014E0007F916F915F914F913F912F910F900FBE20
:1014F0000F901F901895559A89B78F7E89BF0895D0
:10150000CF93DF93DC01EC01EA81FB812091E801BC
:10151000422F5527CA0180739070892B89F044FFB0
:1015200004C083E18CB9206403C081E18CB92F7BB6
:101530002093E8018091E8018F7C8093E80154C0FA
:1015400027FF02C0559850C0ED018A859B85009702
:10155000A9F18091EB01882339F00C9B05C05598C7
:1015600089B7806189BF40C0ED018A859B8501975D
:101570009B878A878091E901882311F0509A01C0E6
:10158000509881918CB9ED018E819F81E817F90700
:1015900011F4EC81FD81ED01FB83EA832A853B8513
:1015A0008C859D8528173907F9F4E889F9893097E2
:1015B00069F08FEFEF3FF807B9F011C05598ED01D2
:1015C0009B878A87E889F989309729F48FEF9FEF05
:1015D000998B888B09C08FEFEF3FF80729F0848142
:1015E0009581019695838483DF91CF910895CF9360
:1015F000DF93DC018091E7019BB1892B8093E701A8
:101600003CB12091E801222361F0333119F455985F
:10161000206804C0313129F4559A2F772093E801CE
:101620005FC0ED014A855B85888599854817590714
:1016300030F08091E70188608093E70151C04F5FEF
:101640005F4F41305105A1F4ED01E889F9893097E8
:1016500029F48FEF9FEF998B888B2AC08FEFEF3F94
:10166000F80731F18481958101969583848320C0A8
:10167000222399F0ED018E859F8548175907C0F008
:1016800026FD16C05D9B05C083E18CB920642F7DCB
:1016900001C020622093E8010BC08091EA018823F9
:1016A00039F0FD01868597854817590708F01A9A81
:1016B000ED91FC91119731931196FC93EE932D913E
:1016C0003C911197ED018E819F812817390729F4EC
:1016D0008C819D8111969C938E93FD015387428747
:1016E000DF91CF9108950FB6F8940F9288EB8AB9E5
:1016F0000F900FBE08950FB6F8940F925798569812
:1017000055980F900FBE8AE00E946D095498539827
:101710000895AF92BF92CF92DF92EF92FF920F9314
:101720001F93CF93DF9389B1C82FDD27809190005D
:101730009927982F8827C82BD92B8091950086FF51
:1017400006C022E0A22EB12CC12CD12C0DC0599B79
:1017500006C098E0A92EB12CC12CD12C05C080E187
:10176000A82EB12CC12CD12C0E94D7097B018C0151
:101770009E01442755272F5F3F4F4F4F5F4FC601B4
:10178000B5010E94F71A9B01AC01C801B7010E9484
:10179000291BCA01B901DF91CF911F910F91FF90D1
:1017A000EF90DF90CF90BF90AF900895EF92FF92AF
:1017B0000F931F937B018C010E947B0B80919500FE
:1017C00086FD11C0599B08C072E0EE0CFF1C001F83
:1017D000111F7A95D1F707C063E0EE0CFF1C001FC4
:1017E000111F6A95D1F70E94D709DC01CB01BC011A
:1017F000CD01A80197010E94291BDA01C9010196B8
:10180000A11DB11DB695A79597958795019789B9A3
:10181000892F9927809390000E94730B80E090E0BD
:101820001F910F91FF90EF900895529B03C089E0A4
:1018300090E008958091950082FF0AC08091950004
:1018400081FF03C088E090E0089587E090E008956C
:101850008091950081FF03C086E090E0089585E0C7
:1018600090E00895CF93C82F0E947B0B52988091EF
:1018700095008D7F80939500809195008B7F80935C
:1018800095008C2F992787309105B1F0883091050C
:101890001CF4069739F015C08830910541F009977E
:1018A00029F00FC080919500826009C0529A809102
:1018B000950082608093950080919500846080936C
:1018C00095000E94730B0E94150C8C1719F08FEF76
:1018D0009FEF02C080E090E0CF9108958091950045
:1018E00099279C012072307085FF0AC08091950075
:1018F00084FF03C081E090E0089582E090E00895C5
:10190000C9010895CF93C82F0E947B0B8C2F992774
:101910008130910591F0823091051CF4892B21F0E2
:101920001AC0029771F017C0809195008F7E809346
:101930009500809195008F7D0CC08091950080610D
:1019400003C0809195008F7E8093950080919500D3
:101950008062809395000E94730B0E946E0C8C171E
:1019600019F08FEF9FEF02C080E090E0CF910895D3
:101970008091950083FF03C082E090E0089581E0AC
:1019800090E00895CF93C82F0E947B0BC13021F4C3
:1019900080919500877F05C0C23029F48091950021
:1019A0008860809395000E94730B0E94B80C8C177E
:1019B00019F08FEF9FEF02C080E090E0CF91089583
:1019C00020E030E040E050E08091E701992784FF7B
:1019D00004C021E030E040E050E083FD226082FD61
:1019E00024608091E801882321F086FD426087FD14
:1019F00048601A9B07C032608091EA01882319F081
:101A0000426001C031600C9B07C038608091EB01DF
:101A1000882319F0426001C0346041FF416043FFF8
:101A200044608091E901882311F0406401C040685E
:101A3000589B02C0406101C04062CA01B9010895CB
:101A4000EF92FF920F931F937B018C018091E8012D
:101A50008823D9F00FB6F8940F9200FF02C08F7B55
:101A600003C001FF03C080648093E80102FF04C04B
:101A70008091E8018F7705C003FF05C08091E801E0
:101A800080688093E8010F900FBE8091EA0188235F
:101A900021F001FD1A9A00FD1A98F1FC1A9AF0FC47
:101AA0001A9806FF03C081E08093E90107FF02C096
:101AB0001092E90104FD589A05FD5898D801C70114
:101AC00081709070A070B070892B29F08091E7012F
:101AD0008F7E8093E701E1FE05C08091E701877F5B
:101AE0008093E701E2FE05C08091E7018B7F809340
:101AF000E7010E94E00CDC01CB01887F8E159F0579
:101B0000A007B10719F08FEF9FEF02C080E090E0CF
:101B10001F910F91FF90EF90089590E080919500B4
:101B200086FF09C091E0129993E08091950080FFB3
:101B300004C0946002C0599990E2892F99270895B2
:101B4000CF93C82F0E947B0B8C2F992780FF13C047
:101B500081FF02C0129A01C0129882FF04C08091D6
:101B60009500816003C0809195008E7F80939500E1
:101B700059985E9A0FC085FF02C0599A01C05998C2
:101B8000809195008E7F80939500809195008F7B4A
:101B9000809395000E94730B0E948D0D8C1719F095
:101BA0008FEF9FEF02C080E090E0CF91089520E09A
:101BB00030E040E050E08091E801882321F020E20D
:101BC00030E040E050E08091EA01882311F021608C
:101BD00001C02E7F8091EB01882311F0226001C0AB
:101BE0002D7FCA01B9010895EF92FF920F931F93C1
:101BF0007B018C0165FF0BC08091E801882371F4A3
:101C00000FB6F8940F9281E48093E80105C00FB6F7
:101C1000F8940F921092E8010F900FBED801C701FF
:101C200081709070A070B070892B31F01A9A129A5E
:101C300081E08093EA0107C08091EA01882319F0CE
:101C40001092EA011298E1FE10C040E050E06BE70C
:101C50007AE08DEB91E00E94041A892BE9F41C9A3A
:101C6000149881E08093EB010EC08091EB018823F2
:101C700051F01092EB0140E050E0BA018DEB91E0A1
:101C80000E94041A14980E94D70DDC01CB018E1516
:101C90009F05A007B10719F08FEF9FEF02C080E00A
:101CA00090E01F910F91FF90EF900895559A08953D
:101CB0009091E8019923A9F096FF13C00FB6F8940C
:101CC0000F925D9B04C081E18CB99F7E01C0906141
:101CD0009093E8018091E8018F798093E8010F905B
:101CE0000FBE8091EA0181111A980895CF93DF9376
:101CF0004AE751E067EF7AE081EB91E00E94041A35
:101D0000EC01892B81F448E651E060E87AE087EB4A
:101D100091E00E94041A009741F0AE01BE0181EBF0
:101D200091E00E94041A8FEF9FEFDF91CF91089509
:101D300040E050E0BA0181EB91E00E94041A40E0DB
:101D400050E0BA0187EB91E00E94041A8091EB0108
:101D5000882351F01092EB01149840E050E0BA0152
:101D60008DEB91E00E94041A8091EA01882319F01A
:101D70001092EA01129880E090E00895CF93DF93EB
:101D8000EA01DC01FB01219724F00E945F1B019214
:101D9000FACF80E090E0DF91CF910895CF93DF9369
:101DA000EC01FB0160E070E06417750790F4DE0160
:101DB000A60FB71F9D010E945F1B802D9081891780
:101DC00021F0D901092E0E94671B31966F5F7F4F6A
:101DD000EBCF80E090E0DF91CF9108959C01FB0173
:101DE00060E070E08AB1482F5527407850705798CE
:101DF00020313105C1F0213131053CF42115310587
:101E000071F02130310561F023C02231310529F113
:101E1000223131050CF120323105A9F019C0AB0196
:101E20008CB18CB117C05F9B05C081E090E09183BD
:101E3000808302C0718360834115510559F0808110
:101E40009181806802C080E190E09183808302C02C
:101E50006FEF7FEF452B09F0579ACB0108951F9242
:101E60000F920FB60F9211242F933F934F935F93CE
:101E70006F937F938F939F93AF93BF93EF93FF9352
:101E800081EB91E00E94F919FF91EF91BF91AF9121
:101E90009F918F917F916F915F914F913F912F9182
:101EA0000F900FBE0F901F9018959C01FB0160E0F2
:101EB00070E08AB1482F55274072507055982131F3
:101EC000310551F1223131053CF42115310529F15B
:101ED0002031310541F01CC022313105F1F02032B2
:101EE000310589F015C05D9B05C081E090E09183CC
:101EF000808302C0718360834115510559F0808150
:101F00009181806802C080E190E09183808302C06B
:101F10006FEF7FEF452B09F0559ACB0108951F9283
:101F20000F920FB60F9211242F933F934F935F930D
:101F30006F937F938F939F93AF93BF93EF93FF9391
:101F400087EB91E00E94F919FF91EF91BF91AF915A
:101F50009F918F917F916F915F914F913F912F91C1
:101F60000F900FBE0F901F9018959C01FB01A0E0F1
:101F7000B0E089B7482F55274071507089B78F7EE0
:101F800089BF2131310509F47DC0223131056CF45E
:101F90002130310519F1223031051CF4232BC1F019
:101FA0006DC020313105E9F069C02831310559F1A2
:101FB000293131052CF42231310509F466C05EC0A7
:101FC00029313105A9F12032310509F452C056C03A
:101FD0008AB78E7F8ABF8AB78D7F8ABF80E188BF2C
:101FE0004FC008B604FE05C081E090E09183808375
:101FF00002C0B183A0834115510509F441C080811D
:102000009181806838C08AB7982F927081FF03C091
:1020100085E090E030C0913019F487E090E02BC06B
:10202000923019F486E090E026C081E090E023C071
:10203000608171816130710519F48AB78E7F05C0A6
:102040006730710531F48AB781608ABF8AB78D7FA6
:102050000EC06530710519F48AB78E7F05C06630F1
:10206000710561F48AB781608ABF8AB782608ABFCE
:1020700007C084E090E09183808302C0AFEFBFEFA0
:10208000452B19F089B7806189BFCD0108951F9252
:102090000F920FB60F9211242F933F934F935F939C
:1020A0006F937F938F939F93AF93BF93EF93FF9320
:1020B0008DEB91E00E94F919FF91EF91BF91AF91E3
:1020C0009F918F917F916F915F914F913F912F9150
:1020D0000F900FBE0F901F901895FC018081918189
:1020E0000895CF92DF92EF92FF920F931F93CF93B9
:1020F000DF936C01CB010E9484117C018F5F9F4FA5
:10210000C9F123E08091C9019091CA01892B61F046
:10211000273050F52F5FE22FFF27EE0FFF1FED5303
:10212000FE4F80819181F2CFC22FDD27CC0FDD1FC2
:10213000CD53DE4F87E090E00E9474118C019983AB
:102140008883009721F1B701C6010E94F310F801BE
:10215000918380838F5F9F4F81F4888199810E9452
:1021600081111982188206C087E190E090933202B3
:102170008093310280E090E00AC0E881F981F38227
:10218000E2821482E881F98116821582CF01DF9103
:10219000CF911F910F91FF90EF90DF90CF90089516
:1021A000FC01CB01DF010D900020E9F71197AE1B78
:1021B000BF0BAD01BF01FC01808191810E946111C3
:1021C0000895CF93DF93EC01AA81BB81109719F496
:1021D000EB85FC8504C0ED01ED89FE89CD010995F3
:1021E000DF91CF910895CF92DF92EF92FF920F93FC
:1021F0001F93CF93DF93CDB7DEB729970FB6F8942F
:10220000DEBF0FBECDBF7B018C0120E0DC018C91D5
:10221000882381F08A3371F0FE0131960F5F1F4FE2
:1022200081932F5FD8018C91882321F08A3311F09C
:102230002830A0F3CE010196FC01E20FF11D1082BF
:102240000E949F01DC01892B49F482E090E0909389
:102250003202809331028FEF9FEF11C0F80181911C
:102260008F018A3311F000E010E0FD01C58CD68C9F
:1022700020E030E0A701B801CD01F60109952996CB
:102280000FB6F894DEBF0FBECDBFDF91CF911F9187
:102290000F91FF90EF90DF90CF900895CF93DF9351
:1022A000DC01EC01EA81FB81309719F4ED81FE81BC
:1022B00003C00788F08DE02DCD010995DF91CF9106
:1022C0000895CF93DF93DC01EC01EA81FB81309725
:1022D00019F4EF81F88503C0018CF28DE02DCD015A
:1022E0000995DF91CF9108950E94EA059C01892B01
:1022F00031F48CE090E09093320280933102C90176
:1023000008950E9470060895FC0140E050E4808129
:10231000282F332727FD30952237310579F02337D1
:10232000310524F42136310539F01FC02737310536
:10233000E1F441E053E402C048E051E43196808189
:102340008823E1F08081282F332727FD30952B3219
:10235000310521F02236310529F007C04E7F426059
:102360005360ECCF5F7B5068E9CF86E190E09093BB
:102370003202809331028FEF9FEF0895CA010895D2
:10238000189A939A8B9A80E00E9473010895089599
:10239000882321F087E00E949312089587E00E942D
:1023A0008612089584B7806884BF84BF089584B777
:1023B0008F7784BF84BF089580919A00877F809330
:1023C0009A008B9893988A9892988C9894981598DC
:1023D0001D98809161008F7B8093610080916200E5
:1023E0008F7B80936200809161008F7D809361007C
:1023F000809162008F7D80936200809161008F7E6A
:1024000080936100809162008F7E809362000895C6
:1024100080919A00886080939A008B9A939A8A9808
:10242000929A8C9A15980895882321F086E00E944C
:10243000861203C086E00E94931283ED91E00E9411
:10244000DC1183ED91E00E94D211089583ED91E0BB
:102450000E94DC1183ED91E00E94D21180E00E9485
:10246000141281E00E94C811089581E00E941412A4
:1024700064EF71E080E090E00E94E10280E00E9461
:10248000C81183ED91E00E94D71183ED91E00E9485
:10249000081260ED77E080E090E00E94E10208958C
:1024A0000E94261268EE73E080E090E00E94E10254
:1024B0000E9435120895882321F085E00E9486123B
:1024C000089585E00E9493120895882321F084E006
:1024D0000E948612089584E00E9493120895282F86
:1024E0000FB6F8940F929927F82FEE2780818083FA
:1024F000C59A0000C5980F900FBE2093EC01089577
:10250000BD9A8091EC010E946F12089521E030E0A5
:1025100002C0220F331F8A95E2F78091EC01822BD3
:102520000E946F12089521E030E002C0220F331F95
:102530008A95E2F7922F90958091EC0189230E9471
:102540006F1208951F93CF93DF9310E0C0E0D0E0A7
:102550008091170299270C2E02C0959587950A94B1
:10256000E2F780FF04C0812F0E94B81A03C0812FB8
:102570000E94C61A1F5F2196143050F3DF91CF914D
:102580001F910895CF93DF93C82FDD27C0FF04C0AC
:1025900080E00E94B81A03C080E00E94C61AC1FF02
:1025A00004C081E00E94B81A03C081E00E94C61AEC
:1025B000C2FF04C082E00E94B81A03C082E00E94F9
:1025C000C61AC3FF04C083E00E94B81A03C083E0A8
:1025D0000E94C61ADF91CF910895562F622F9091D5
:1025E0002F02292F3327F901EE0FFF1FEE0FFF1FD8
:1025F000E75EFD4F8083518342836383C901019667
:1026000065E070E00E94161B80932F02982F809146
:102610001802981749F4892F9927019665E070E010
:102620000E94161B809318020895C0E086E90E945C
:102630008C05E091180280912F02E81719F410928E
:102640002D0221C0FF27EE0FFF1FEE0FFF1FE75ED9
:10265000FD4F808180932D0210E0812F0E94C61AC9
:102660001F5F1430D0F380911802E82FFF27EE0F80
:10267000FF1FEE0FFF1FE75EFD4F83818F3F11F0BD
:1026800081508383C28180912D02992784309105E6
:1026900009F48DC08530910594F48130910509F4D9
:1026A00057C0823091051CF4892BC9F079C1823062
:1026B000910509F465C0039709F4A6C071C186307D
:1026C000910509F4E3C0863091050CF4C0C0873051
:1026D000910509F4FCC0089709F434C161C18091E7
:1026E000D401882359F10E9465157B018C019091DA
:1026F000D5018FE3989FC00111249C0144275527E1
:10270000C801B7010E94291BDC01CB01CF97A105AD
:10271000B105A0F46091ED01662321F021E0409124
:10272000D40107C080911702882331F421E0422FA1
:10273000622F84E00E94ED1210922E0280912E02F0
:102740008F5F80932E026FE370E080E090E025C100
:1027500080911802E82FFF27EE0FFF1FEE0FFF1FDB
:10276000E75EFD4F81810E94C2128FE3C89FC001C6
:102770001124AA2797FDA095BA2FBC01CD010DC148
:1027800080911802E82FFF27EE0FFF1FEE0FFF1FAB
:10279000E75EFD4F81810E94C2128FE3C89FC00196
:1027A00011247C010027F7FC0095102F22C080E047
:1027B0000E94C2128FE3C89FC00111247C01002730
:1027C000F7FC0095102FC801B7010E94E10280912B
:1027D0002D02882309F4EFC080911802E82FFF270B
:1027E000EE0FFF1FEE0FFF1FE75EFD4F81810E947E
:1027F000C212C801B7010E94E10280912D02882314
:1028000009F4D9C080E020C080E00E94C2128FE3AA
:10281000C89FC00111247C010027F7FC0095102FF0
:10282000C801B7010E94E10280912D02882309F4BA
:10283000C2C080911802E82FFF27EE0FFF1FEE0F96
:10284000FF1FE75EFD4F81810E94C212A4C080E09D
:102850000E94B81A10E08FE3C89FC00111246C01D8
:10286000EE24D7FCE094FE2CC701B6010E94E102E1
:1028700080912D02882341F1812F0E94C61A1F5F8B
:10288000812F0E94B81A133030F31EC083E00E94DB
:10289000B81A13E08FE3C89FC00111246C01EE2425
:1028A000D7FCE094FE2CC701B6010E94E1028091A2
:1028B0002D02882349F0812F0E94C61A1150812FC2
:1028C0000E94B81A112331F7C701B60166C080E033
:1028D0000E94B81A10E08FE3C89FC00111249C0128
:1028E000442737FD4095542FCA01B9010E94E102E7
:1028F00080912D02882349F0812F0E94C61A1F5F04
:10290000812F0E94B81A133030F313E08FE3C89F71
:10291000C00111249C01442737FD4095542FCA0162
:10292000B9010E94E10280912D02882309F443C07D
:10293000812F0E94C61A1150812F0E94B81A1123AC
:1029400029F739C080E00E94B81A81E00E94B81AC5
:1029500082E00E94C61A83E00E94C61A8FE3C89FD5
:10296000C00111247C010027F7FC0095102FC8013D
:10297000B7010E94E10280912D028823E1F080E0FE
:102980000E94C61A81E00E94C61A82E00E94B81A0C
:1029900083E00E94B81AC801B7010E94E1020BC08F
:1029A00080911802E82FFF27EE0FFF1FEE0FFF1F89
:1029B000E75EFD4F138280912D02882309F439CE02
:1029C00080911802282F3327F901EE0FFF1FEE0F19
:1029D000FF1FE75EFD4F8381882309F02ACEC901DE
:1029E000019665E070E00E94161B20912F023327AC
:1029F0008217930711F40E94A2128091180299275E
:102A0000019665E070E00E94161B8093180211CEBB
:102A100080912F02809318020E94A21210922D0220
:102A200008958093D5016093ED014093D4010895FA
:102A30001F93182F0E94D41A10922F02109218027E
:102A4000112351F020E034E040E050E065E173E113
:102A500086ED91E00E94D4081F910895CF93C82F6E
:102A600080912D02882319F48C2F0E94B81A81E0DE
:102A700090E002C0880F991FCA95E2F720911702D3
:102A8000282B20931702CF910895CF93C82F8091C0
:102A90002D02882319F48C2F0E94C61A81E090E041
:102AA00002C0880F991FCA95E2F7982F90958091E0
:102AB0001702892380931702CF9108950E9408047A
:102AC000DC01CB01BC01CD01089580913002813041
:102AD00089F40E9408049B01AC018091EE01909161
:102AE000EF01A091F001B091F101280F391F4A1FA9
:102AF0005B1F10C00E9408049B01AC018091EE0195
:102B00009091EF01A091F001B091F101281B390BD8
:102B10004A0B5B0BCA01B9010895DC01CB0180931C
:102B2000EE019093EF01A093F001B093F101409377
:102B3000300208950F931F93CF93DF93FC01C18957
:102B4000D289EDA9FEA909958C01892B49F4CF5BA7
:102B5000DF4FE881F98160E072EC81E090E0099557
:102B6000C801DF91CF911F910F910895AF92BF924D
:102B7000CF92DF92EF92FF920F931F93CF93DF9349
:102B80008C017B016A015901FC01C481D5818085DA
:102B900091850FB6F8940F92118610860F900FBE94
:102BA0008617970799F0892B29F0209719F0CE0105
:102BB0000E948111E114F10449F0C7010E947411CF
:102BC000EC01892B19F48FEF9FEF1DC0E114F10484
:102BD000C1F0F801D583C483D183C083D383C2837A
:102BE000CE0DDF1DD783C683D586C486B786A6865D
:102BF000138612860FB6F8940F92F186E0860F9036
:102C00000FBE80E090E0DF91CF911F910F91FF9078
:102C1000EF90DF90CF90BF90AF9008956F927F922A
:102C20008F929F92AF92BF92CF92DF92EF92FF92DC
:102C30000F931F93CF93DF939B013A01882499242C
:102C40007B01EC01EA81FB8101891289E801A296EE
:102C5000688579856115710519F48FEF9FEFA5C01F
:102C6000232B69F42E853F854C855D85CE010E941E
:102C7000B615E801EBADFCAD0995C40196C00FB6E1
:102C8000F8940F92AA84BB840F900FBEA114B104D4
:102C900091F4F80183AD94ADFC010995F8014085EC
:102CA000518562857385CE0140960E947607892BF7
:102CB00031F3C5017AC0F801808187FF39C0CC2487
:102CC000DD24C614D70408F06FC05AE08A149B04B0
:102CD00008F051C0EA81FB814191FB83EA832A819C
:102CE0003B818E819F812817390721F48C819D813A
:102CF0009B838A830894811C911C4D3011F04A30CB
:102D000059F4F80184A9882311F0841769F4F801B3
:102D100044ABF701519304C0F80114AAF7014193A1
:102D20007F010894C11CD11CC614D70478F223C0BB
:102D30006301A614B70408F46501882499248C144F
:102D40009D0490F5EA81FB818191FB83EA83F70181
:102D500081937F012A813B818E819F8128173907CA
:102D600021F48C819D819B838A830894811C911C12
:102D70008C149D0438F381149104B1F00FB6F894CB
:102D80000F928A859B85881999099B878A870F905E
:102D90000FBE2A853B858C859D852817390720F431
:102DA000E801EBADFCAD0995C601DF91CF911F9114
:102DB0000F91FF90EF90DF90CF90BF90AF909F90DA
:102DC0008F907F906F900895CF92DF92EF92FF9255
:102DD0000F931F93CF93DF937C016A018C01005FF7
:102DE0001F4F0FB6F8940F92F80182859385860FD6
:102DF000971F93878287C285D3850F900FBECC160D
:102E0000DD06A8F4F70181AD92ADFC010995F7014B
:102E10004485558566857785C80140960E9476076A
:102E2000892B29F40FB6F8940F92F801E4CFCE0164
:102E3000DF91CF911F910F91FF90EF90DF90CF9096
:102E400008956F927F928F929F92AF92BF92CF928E
:102E5000DF92EF92FF920F931F93CF93DF93FB01CB
:102E60004A013901EC01E988FA88E7016096888512
:102E70009985892B19F48FEF9FEF87C06115710534
:102E800029F4AB01C7010E94E4167FC0D7012D9140
:102E90003D914D915C9131FF03C041E0A42E01C0F2
:102EA000AA24D7018C91807819F031E0B32E01C0AB
:102EB000B82E0FB6F8940F924A855B850F900FBE1F
:102EC0008F01CC24DD24B601C814D9040CF05CC0F9
:102ED0009A01260F371F8E859F852817390770F0B6
:102EE0004C855D85C7010E94E416AC0160E070E08E
:102EF0008C859D858417950708F446C0611471047C
:102F000019F0F801849102C0D8018C91B1E0BB1690
:102F100049F48A3061F422E0B22E8DE0AB1661F400
:102F2000AB2C0AC0E2E0BE1611F491E0B92E0F5F9F
:102F30001F4F0894C11CD11CE881F9818193F9834A
:102F4000E883288139818E819F812817390721F4F0
:102F50008C819D81998388836F5F7F4FC814D904CA
:102F60000CF4B6CF6115710579F00FB6F8940F9295
:102F70008A859B85860F971F9B878A870F900FBE38
:102F8000E701E9ADFAAD0995C601DF91CF911F9137
:102F90000F91FF90EF90DF90CF90BF90AF909F90F8
:102FA0008F907F906F90089520E030E0FC01828147
:102FB00093810E942117089521E030E0FC01828175
:102FC00093810E9421170895CF93DF93DC01EC01D8
:102FD000EA81FB81C189D289892B21F08FEFAF3F34
:102FE000B80719F48FEF9FEF15C0CD010E94811132
:102FF00020E030E0A901B901CE0140960E94B6154B
:1030000020E030E0A901B901CE0182960E94B615F8
:1030100080E090E0DF91CF910895CF92DF92EF9220
:10302000FF920F931F93CF93DF936C017A01FC0102
:10303000C189D289CA0183709070892B61F02EE119
:1030400030E044E150E060E270E0CE0140960E9442
:10305000B615892B19F5C70183709070019779F027
:103060002EE130E044E150E060E270E0CE01829673
:103070000E94B615892B19F08C899D890DC086E0B8
:1030800090E00E9474118C01892B59F48C899D89E0
:103090000E9481118EA19FA10E9481118FEF9FEF4D
:1030A00023C0C7018070907C288139814A815B816F
:1030B0008050904811F42F7701C02068288339830D
:1030C0004A835B83F80111821082D382C282158207
:1030D0001482F3E0EF22FF2461E0E616F10419F018
:1030E000EBADFCAD0995C801DF91CF911F910F9118
:1030F000FF90EF90DF90CF900895AF92BF92CF9264
:10310000DF92EF92FF920F931F93CF93DF936A01A9
:10311000AA24BB24DA01ED90FD900D911C912E2D77
:10312000FC01C189D289615071406732710508F094
:103130003AC16A5B7F4FFB01EE0FFF1F0590F491D0
:10314000E02D0994CF5BDF4F4BC0CD5BDF4FA8C0B4
:10315000CB5BDF4F05C0C95BDF4FCDC0C75BDF4F27
:10316000E881F981822F0995ECC0C55BDF4FC3C0B0
:10317000C35BDF4FF5CFC15BDF4FBDC0E6FE11C0C3
:10318000FE01B29626853785448555856085718513
:10319000CF010E94B6155C01892B19F4EBADFCAD93
:1031A0000995E7FE0FC0FE017096A114B10451F419
:1031B000268537854485558560857185CF010E94B8
:1031C000B6155C01A114B10409F0F0C0CF5ADF4F6D
:1031D0008FE39FEFAFEFBFEFE822F9220A231B2313
:1031E000E881F981C801B7010995ABC0CD5ADF4F1D
:1031F000E881F981C355D04009959B01AC01D60106
:103200006D937D938D939C9313978CA59DA5892B8E
:1032100031F42064F60120833183428353838A8D05
:103220009B8D892B09F0C2C0F60180819181A2811A
:10323000B3818068B3C0E886F9860A871B87B6C069
:1032400088859985AA85BB85A8C0EC86FD860E87F2
:103250001F87ACC08C859D85AE85BF859EC088814B
:103260009981AA81BB81EE2011F0806428C08F7BF8
:1032700026C088819981AA81BB819C01AD012074FF
:1032800030704070507086FD22C0D6012D933D9362
:103290004D935C9313978AC0EDADFEADA3CFEF962F
:1032A000E881F9810995DC01CB0177C0888199819A
:1032B000AA81BB81EE2011F0806801C08F778883DE
:1032C0009983AA83BB8372C0888187FF05C081E090
:1032D00090E0A0E0B0E061C0DA011D921D921D9265
:1032E0001C92139763C0CB5ADF4FE881F9818E2D72
:1032F0003ACFC95ADF4FE881F98109959927AA2762
:10330000BB274BC0FE0170962685378544855585C1
:10331000B701CF010E94B6155C01892B09F046C0A8
:10332000EBADFCAD099542C0888D998D34C0FE018E
:10333000B2962685378544855585B701CF010E9411
:10334000B6155C0133C08AA59BA525C00FB6F894BD
:103350000F92FD8EEC8E1AC08C8D9D8D1CC00FB609
:10336000F8940F92FF8EEE8E11C08E8D9F8D13C03C
:103370000FB6F8940F92FFA6EEA608C08EA59FA5E3
:103380000AC00FB6F8940F92F9AAE8AA0F900FBEE0
:103390000DC088A999A9AA27BB27F601808391832C
:1033A000A283B38303C05FEFA52EB52EC501DF91C5
:1033B000CF911F910F91FF90EF90DF90CF90BF9032
:1033C000AF900895CF93DF93EC01EA81FB810188F0
:1033D000F289E02DB2960FB6F8940F92828593850C
:1033E000AA27BB270F900FBEBC01CD01DF91CF9163
:1033F0000895FC01228133812115310521F080815E
:103400009181F90109950895EF92FF920F931F930F
:10341000CF93DF93EC017B018A0180E090E0EC81A7
:10342000FD81309711F0BC01099519830883FB8257
:10343000EA82DF91CF911F910F91FF90EF90089555
:10344000CF93DF932FEF3FEFEC01EC81FD813097BD
:1034500031F060E070E081E190E009959C01C901E4
:10346000DF91CF910895CF93DF932FEF3FEFEC01E2
:10347000EC81FD81309731F060E070E082E190E016
:1034800009959C01C901DF91CF9108950F931F9376
:10349000CF93DF93CDB7DEB724970FB6F894DEBF96
:1034A0000FBECDBF8C017C836B838FEF9FEFF80144
:1034B0002481358121153105B9F0BE016F5F7F4F41
:1034C00080E290E0F9010995009771F4F8012481F8
:1034D0003581BE016D5F7F4F81E290E0F901099572
:1034E000009711F489819A8124960FB6F894DEBF73
:1034F0000FBECDBFDF91CF911F910F9108950F9314
:103500001F93CF93DF93CDB7DEB724970FB6F89410
:10351000DEBF0FBECDBF8C017C836B838FEF9FEF2F
:10352000F8012481358121153105B9F0BE016F5FA5
:103530007F4F88E190E0F9010995009771F4F80157
:1035400024813581BE016D5F7F4F89E190E0F901F3
:103550000995009711F489819A8124960FB6F89401
:10356000DEBF0FBECDBFDF91CF911F910F910895A8
:10357000882321F0813011F0823019F40E948612E4
:103580000895833011F40E9486120895882321F053
:10359000813011F0823019F40E9493120895833023
:1035A00011F40E94931208950E94801280E00E94FC
:1035B000C61A81E00E94C61A82E00E94C61A83E001
:1035C0000E94C61A0895DC0140FF03C001C06D933C
:1035D0006D9342505040D8F70895FB01DC018D9166
:1035E0000190801911F40020D1F7990B0895629F82
:1035F000D001739FF001829FE00DF11D649FE00DEB
:10360000F11D929FF00D839FF00D749FF00D659F4B
:10361000F00D9927729FB00DE11DF91F639FB00D4A
:10362000E11DF91FBD01CF011124089597FB092E5B
:1036300007260AD077FD04D02ED006D000201AF439
:10364000709561957F4F0895F6F7909581959F4FFE
:103650000895A1E21A2EAA1BBB1BFD010DC0AA1FD3
:10366000BB1FEE1FFF1FA217B307E407F50720F0EB
:10367000A21BB30BE40BF50B661F771F881F991F66
:103680001A9469F760957095809590959B01AC01AF
:10369000BD01CF010895AA1BBB1B51E107C0AA1FA2
:1036A000BB1FA617B70710F0A61BB70B881F991FE3
:1036B0005A95A9F780959095BC01CD010895E1999F
:1036C000FECFBFBBAEBBE09A11960DB20895E19953
:1036D000FECFBFBBAEBB0DBA11960FB6F894E29AFF
:0636E000E19A0FBE0895FF
:1036E600722B00554152542D6563686F20617070CE
:1036F6006C69636174696F6E210A00FF6D61696EA2
:103706000065746865726E75740069646C650000A6
:103716000000000F0A00007561727430000000009E
:1037260005000000000058019A157D180E16D417E2
:10373600DC170D18E417E219000000000000000075
:103746000000000000000000000000000000000073
:103756000000000000000000000000000000000063
:1037660000000000000000000000000000760E9837
:103776000E560E580EF40DD70DD60B890B320C15BE
:103786000C820C6E0CC20CB80C200DE00CA00D8D3A
:103796000D00000000EE0E00000000550F000000B6
:1037A60000B50F0100020003000000000000000049
:0A37B60000000000010F4C45440024
:00000001FF
